:020000020000FC
:10000000A895DFE0D1BDDFEED7BBD0EFD8BBD0E005
:10001000D5BFEE246627442725D165FF14C0D5D06F
:100020000CD1D0E08D2F712DC9D0D1E08D2F702D46
:10003000C5D028D1D0EFD8BBA8950AD134D14AD1A8
:1000400012D081D0F9CF77278827A895B49BFFCF0E
:1000500073957F3FE8F383958031D0F37727882726
:100060004F6071D0F2CFC72DD62DDF19C50B68F0C8
:10007000C52DD42DDF19C50B08F40EC0677F3324BE
:1000800062FD089564608A940895677F332461FD5A
:1000900008956260839408956D7F6B7F63FD08957A
:1000A000D32DD03310F43394089563FD0895D82DE3
:1000B000D33899F0DF3759F1D138D9F0D23899F0E7
:1000C000DE3799F1DD3739F0DC3719F0D0E88D2EC5
:1000D00008954F6135C0407E33C042FD02C0446088
:1000E00001C04B7F2DC043FD02C0486001C0477F67
:1000F00027C022E344FD4D7F41FD05C022E34E7F32
:100100004F7E426003C04D7F4E7F4F7E19C022E379
:1001100044FD4E7F40FD05C022E341604F7E4D7F90
:1001200003C04E7F4F7E4D7F0BC044FD05C02EE1C6
:1001300040614160426003C04F7E4E7F4D7F00C0F2
:10014000D0E88D2E089542FD02C0C19801C0C19A29
:100150002395223308F022272E3120F000C0C098CA
:10016000C29809C041FFC09840FFC29841FDC09AA3
:1001700040FDC29A00C043FF09C09395923020F021
:10018000903120F0992704C0C39A02C0C39800C0E0
:1001900043FF0AC0E395E23020F0E13128F0EE277A
:1001A00006C0DFEED7BB03C0DFECD7BB00C00895AD
:1001B0008EBBE09AE099FECF7DB308957DBB8EBBE8
:1001C000E29AE19AE199FECF0895AA24BB2440D097
:1001D0003FD03ED03DD03CD0AB0EBA1E39D0AB0E96
:1001E000BA1E36D0AB0EBA1E33D0AB0EBA1E30D00C
:1001F000AB0EBA1E2DD0AB0EBA1E2AD0AB0EBA1E55
:1002000027D0AB0EBA1E089523D0AB0EBA1E20D055
:10021000AB0EBA1E1DD0AB0EBA1E1AD0AB0EBA1E54
:1002200017D0AB0EBA1E14D0AB0EBA1E11D0AB0E47
:10023000BA1E0ED0AB0EBA1E08951A2C0B2C0694C3
:1002400017940694179406941794C12CD02C0895F3
:10025000BB27AA27D1E0B49BFECFBD0FAE1DB4993A
:10026000FCCF08956062BB27AA27D1E0B49BFECFE4
:10027000BD0FAE1DCA2FC03818F4B499F9CF089538
:100280006F7D08954424552466247724412C502CF6
:10029000612C702CD2E36D0E7E1C4D1A5E086860D6
:1002A000D0E88D2E0895012D102D02581E09DB2F48
:1002B000CA2FD01BC10B58F0012D102DD2E80D0F05
:1002C0001E1DDB2FCA2FD01BC10B08F40895BC2DB7
:1002D000AD2D0895AB0EBA1EFA2C5B2D5695F794F2
:1002E0005695F7945695F794AF18B50ACF2CD52E9E
:0202F00008956F
:00000001FF
